:020000040800F2
:10000000807E002085010008731100085F0D000844
:100010007111000869020008F115000800000000D5
:100020000000000000000000000000005D13000858
:100030006B02000800000000751100085914000848
:100040009F0100089F0100089F0100089F01000810
:100050009F0100089F0100089F0100089F01000800
:100060009F0100089F0100089F0100089F010008F0
:100070009F0100089F0100089F0100089F010008E0
:100080009F0100089F0100089F0100089F010008D0
:100090009F0100089F0100089F0100089F010008C0
:1000A0009F0100089F0100089F0100089F010008B0
:1000B0009F0100089F0100089F0100089F010008A0
:1000C0009F0100089F0100089F0100089F01000890
:1000D0009F0100089F0100089F0100089F01000880
:1000E0009F0100089F0100089F0100080000000018
:1000F0000000000000000000000000000000000000
:1001000000000000000000009F0100089F0100089F
:100110009F0100089F0100089F0100089F0100083F
:100120009F0100089F0100089F0100089F0100082F
:100130009F0100089F0100089F0100089F0100081F
:100140009F0100089F0100089F0100089F0100080F
:10015000DFF80CD000F076F800480047753700084B
:10016000807E0020EFF30980704780F30988704794
:10017000EFF30880704780F30888704740BA7047F3
:10018000C0BA70470648804706480047FEE7FEE7CA
:10019000FEE7FEE7FEE7FEE7FEE7FEE7FEE7FEE737
:1001A0005D1400085101000840EA01039B0703D0D9
:1001B00009E008C9121F08C0042AFAD203E011F8A6
:1001C000013B00F8013B521EF9D27047D2B201E068
:1001D00000F8012B491EFBD270470022F6E710B54C
:1001E00013460A4604461946FFF7F0FF204610BDA5
:1001F00010B5044604E00B7800F8013B03B1491C3C
:10020000521EF8D2204610BD421C10F8011B0029D6
:10021000FBD1801A704730B50B46014600202022E2
:10022000012409E021FA02F59D4205D303FA02F503
:10023000491B04FA02F52844151EA2F10102F1DC63
:1002400030BD0000064C074D06E0E06840F00103B9
:1002500094E8070098471034AC42F6D3FFF77CFFD0
:100260007043000890430008FEE77047FEB5012187
:10027000084600F099FF0121022000F095FF144D7F
:100280000124ADF80440286812490026B0FBF1F0C3
:10029000401EADF800001027ADF80660ADF8027002
:1002A0006946A00701F04EF9ADF8044028684FF404
:1002B000FA61B0FBF1F0401EADF80000ADF8066049
:1002C000ADF802706946044801F03CF9FEBD00003B
:1002D000A000002080841E0000040040F1B5424CC4
:1002E0008CB00C986169401AFA2832D30C983F4DB3
:1002F0006061A0686968012681422CD0012003F06A
:1003000079F9032001F07CFA6868A060070EC0F359
:100310000741CDE90017C0F30723C2B234A102A8F8
:1003200001F068F902A9012000F0B4FEA868A060FD
:10033000050EC0F30741CDE90015C0F30723C2B293
:100340002FA102A801F056F902A9022000F0A2FE96
:1003500026700DB0F0BD0028FBD1286A4078042833
:10036000F7D9224802F034F82A4802F022FC08901B
:100370006FF0FF0002F01DFC09902648093802F0DA
:1003800018FC0A90012003F035F9032001F038FA37
:100390000898A060050EC0F30741CDE90015C0F331
:1003A0000723C2B212A102A801F024F902A9012078
:1003B00000F070FE0998A060050EC0F30741CDE97A
:1003C0000015C0F30723C2B20DA102A801F012F973
:1003D00002A9022000F05EFE26700AAB09AA08A955
:1003E000024803F052FBB4E710000020B4000020E4
:1003F00049503A25642E25642E25642E256400007C
:100400004D41534B3A25642E25642E25642E2564D8
:10041000000000000A00A8C005490028886902D031
:1004200040F0020001E020F0020088617047000007
:1004300000900240F0B5104C00234FF0004644F20B
:10044000F057551E606012E0C3EB431C00EB031431
:100450000CEB831C01EB0C1C84E8C010AB4204D2F3
:1004600004F1100CC4F80CC000E0E0605B1C934287
:10047000EAD30249C860F0BD480000200090024065
:1004800005490028886902D040F4005001E020F4BA
:10049000005088617047000000900240F0B50F4C9A
:1004A00000234FF48016551E206011E0C3EB431764
:1004B00000EB031407EB831701EB0717A760266017
:1004C000AB4203D204F11007E76000E0E0605B1C80
:1004D0009342EBD302490861F0BD000048000020C0
:1004E0000090024002680A430260704710B5012183
:1004F0008C03204600F04CFE2046BDE81040002151
:1005000000F046BE01B581B001980090002801D0EE
:10051000401EFAE70CBD00000248816941F48011D9
:100520008161704700900240014800688068704710
:1005300048000020064900204968096811F0802F12
:1005400005D1CA0503D58A0501D5C1F30D40704711
:1005500048000020034900200968C90700D0012095
:1005600070470000009002402DE9F04188B000265D
:10057000764D0446009606962869884620F01C07AA
:1005800001A800F029FE72490298724A0144914282
:1005900002D247F0080706E06F4908446F498842D5
:1005A00001D247F00C072F614FF400420021404672
:1005B00000F0D4F900282DD06948FFF7A3FF206888
:1005C000B0B3684F06980121401C0690404600F0E9
:1005D000FBF8400702D40698B842F3D30698B84215
:1005E00017D04FF4805200214046069600F0B6F92D
:1005F00000280FD006980121401C0690404600F0CC
:10060000E3F8800602D40698B842F3D30698B842BD
:1006100003D1002008B0BDE8F081102140460696C5
:1006200000F0D2F8410704D54FF40061216201E0E7
:1006300008E02662800701D5666113E04FF4804030
:1006400060610FE0206A6169C00840EA510082B22F
:100650000021404600F082F90028DBD06FF07F4097
:10066000FFF750FF296840480140D4E901021043D8
:10067000E26854F8103F1A43104362681043A268BE
:100680001043E26810432269104362691043A26973
:100690001043E2691043226A1043626A1043084320
:1006A00028602834D4E900010843D4E90212114338
:1006B00008432169084361690843A1690843E16966
:1006C00008436860206AA860606AE860A9694FF61C
:1006D00041700140D4E90B021043238D626B42EA62
:1006E00003421043A26B1043E26B10430843A8611E
:1006F000D4E910010843E8611C4A91691C48014093
:10070000D4E912031843D4E914352B431843A36DDD
:100710001843E36D1843236E1843636E1843A36EAA
:10072000184308439061D4E91B010843616F54F8F2
:10073000783F19430843616840EA8100A168084393
:1007400040F400001060012064E7000000800240D7
:1007500000D3CEFEC0E1E40040F1E9FD40787D0128
:10076000FFFF0F00FFFF04000F8120FF00900240F9
:10077000233FDEF8054B8A88184402640A78D1F8D2
:10078000011042EA012141647047000000800240EC
:1007900005490028086802D040F0040001E020F07C
:1007A00004000860704700000080024005490028EE
:1007B000086802D040F0080001E020F0080008605E
:1007C000704700000080024018B500220092124AD3
:1007D00013694FF6FF7403F01C0304EAC0201843AA
:1007E0004FF4F86303EA8111014321F0020040F065
:1007F0000100106109480099491C00911169C9075D
:1008000002D000998142F6D30099814201D10020A3
:1008100018BD506980B218BD00800240FFFF04007F
:1008200070B5114D002319462A681468002C0BDAA4
:100830000E4A0B465469240602D580245461936005
:1008400001604160816070BD260407D4E60505D5CE
:10085000A60503D5C4F30D4391681B1FD4682C6013
:100860000360C0E9011270BD4C00002000900240FE
:100870000248016841F001010160704700900240A8
:1008800000B50120FFF792FFFFF746FE0120FFF7BA
:100890007FFF0120FFF7F4FD01205DF804EBFFF777
:1008A000BBBD0021016041608160C16001614161A7
:1008B0008161C161016241628162C1620163416320
:1008C00040228163C0E90F122022C0E91121C164D6
:1008D0000165416581658022C165C0E918128166A4
:1008E000C16601674167D2048167C0E91F125210D7
:1008F0005310C0E921231311C0E92331C0F894102B
:10090000C0F89810C0F89C10C0E928121212C0E973
:100910002A125212C0E92C21C0F8B810704700000A
:100920000C4A11680B68002B01DA00207047C0F3F5
:100930000C00486043F030400860074843695B079B
:1009400003D50423436100234360C868106001207D
:1009500070470000480000200090024038B5002396
:100960000093114B1C694FF6FF7504F01C0405EA57
:10097000C02020434FF4F86404EA8111014341F0A0
:1009800003005A61186109480099491C00911969CE
:10099000C90702D000998142F6D30099814201D162
:1009A000002038BD012038BD00800240FFFF040058
:1009B00000B5AFB0012000F045F94FF4004000F061
:1009C00093FC012000F08AFC3D2000F069FC002827
:1009D000FAD00B2000F07CFCFFF788FDFFF748FF02
:1009E000FFF7B8FD0128FBD06846FFF75AFF01204A
:1009F000009000204FF40071CDE90A10090407901F
:100A00001190CDE920010E90149013900A111590C9
:100A10002590269023920420CDE9280180032A9076
:100A200080012B9040122C9040002E9001216846AE
:100A3000FFF79AFD2FB000BD70B505464FF4302684
:100A4000304600F095F8042813D10A4C206940F094
:100A5000020020616561206940F04000206130465D
:100A600000F086F8052804D0216941F6FD72114096
:100A7000216170BD0020024008490420CA68D207E5
:100A800001D001207047CA68520701D50220704783
:100A9000C968C906FBD5032070470000002002404A
:100AA00070B50446074D09E02046FFF7C5FF04284E
:100AB00002D04FF0FF3070BD04F50064AC42F3D9B2
:100AC000002070BD00F0030800F046B82DE9F041A9
:100AD0001646884605460024094F0DE02868B842AE
:100AE0000CD858F82410286800F00CF8042805D118
:100AF0002868001D2860641CB442EFD3BDE8F08173
:100B0000FBF703082DE9F841064600204FF4005793
:100B100000900D46384600F02BF8042818D10D4CF3
:100B2000206940F0010020613580B846384600F069
:100B30001FF8BF1E042806D1B61C280C0096308072
:100B4000404600F015F8052802D02169394021619E
:100B5000BDE8F88100200240034802494160034992
:100B6000416070472301674500200240AB89EFCD0B
:100B700000B50346FFF780FF03E000BFFFF77CFFEF
:100B80005B1E012803D0002B00D1052000BD002BE7
:100B9000F4D1FAE72DE9F8430426ADF80060032408
:100BA000DFF890808DF8024018258DF803506946D3
:100BB000404600F04DF80227ADF800708DF8024075
:100BC0008DF8035069461C4800F042F84FF460501D
:100BD000ADF800008DF802408DF8035069461748C3
:100BE00000F036F801214FF0201000F081F8ADF848
:100BF00000708DF802408DF803606946404600F0B1
:100C000027F84FF4E060ADF800008DF802408DF851
:100C1000036069460A4800F01BF8B001ADF8000017
:100C20008DF802408DF803506946404600F010F8F8
:100C3000BDE8F8830008014000100140000C0140AD
:100C4000001401400149086070470000DC002042A8
:100C5000F0B5CA78002502F00F03D20601D58A78D4
:100C600013430C784FF00F0E0122ECB1D0F8004086
:100C70000F8802FA05F63740B74211D14FEA850CCA
:100C80000EFA0CF724EA070703FA0CF43C43CF787A
:100C9000282F02D0482F02D002E0466100E0066112
:100CA0006D1C082DE4D304600C88FF2C1ED9446809
:100CB0005FF0000606F1080702FA07F50F882F40DB
:100CC000AF420FD14FEA860C0EFA0CF7BC4303FA81
:100CD0000CF73C43CF78282F00D14561CF78482FBF
:100CE00000D10561761C082EE4D34460F0BD0000FD
:100CF000F0B5144C002801DAE36900E06368420DA6
:100D0000120185B2C0F301579540C0F30346032F8B
:100D100005D0C2020AD50322B240934307E023F074
:100D20007062636823F07063636002E0AB4343F07A
:100D3000706201B12A43002801DAE261F0BD62600D
:100D4000F0BD0000000001400246002092680A4207
:100D500000D0012070474161704701617047FEE794
:100D600010B50446084602F039FD204603F024F988
:100D7000204603F005FA0548002203498068BDE8D3
:100D8000104003F0FAB90000390E000828000020D6
:100D9000408802F0B4BE00002DE9F04781461646B7
:100DA00088464FF40A7002F049FD04002CD002205E
:100DB0002060D8F80000C4F80C020025C4E984655E
:100DC000224614494846C4F8185203F0D6F9124F87
:100DD0003D60FFF779FE114D2846FFF761FE7D600B
:100DE000324641464846D4F8143200F07DF80120DE
:100DF00002F000FC032000F003FD09A1012000F037
:100E000049F90020BDE8F08701464846FFF7A8FFF2
:100E1000F7E70000750F0008280000200090000888
:100E200053746174653A2050726F6772616D6D69B9
:100E30006E672E2E000000002DE9F0438BB098461F
:100E40001746DDF8489003F08BF9060034D00022F5
:100E50001B4903F05DF800282ED17C6860780228D9
:100E600003D0304603F08CF923E0A41C002500E0F9
:100E70006D1C605D0028FBD1012002F0BBFB03204C
:100E800000F0BEFC6A1C214606A8FFF7B1F906AACD
:100E90000CA1684600F0AEFB6946012000F0FAF8AC
:100EA0000CA1022000F0F6F84A4641463046FFF712
:100EB00073FF384602F04FFF0BB0BDE8F08300002F
:100EC0005C4300085570646174652046696C653A3E
:100ED0002573000053746174653A2045726173692B
:100EE0006E672E2E2E0000002DE9F0410E46804642
:100EF0000021042061F3070460F30F24154698B223
:100F000001F059FE60F31F4403220421002002F087
:100F1000F8FD07000ED07868ABB23246046039465F
:100F2000404603F043F90446384602F014FF2046D9
:100F3000BDE8F0814FF0FF30FAE7000010B503F094
:100F40000FF9094C0028A0600CD04522074902F097
:100F5000DFFF002806D1A068BDE810400022044948
:100F600003F00BB910BD0000280000205C4300080E
:100F7000390E00082DE9F043ADF5077D884604469B
:100F800050891189DDF838921F461546884263D191
:100F9000354E042830D96868FFF7FAFED4F81412E9
:100FA000491C884228D168890423001F82B26946FF
:100FB000284602F09CFE69893068001F08443060B2
:100FC000081FC21700EB9270C0F38F02880701D090
:100FD000521C92B224486946001DFFF777FDD4F8F1
:100FE0001402401CC4F814026989D4F81802084499
:100FF000001FC4F818020AE06868FFF7C9FE01463E
:10100000D4F81402401C814201D1C4F814024A46AB
:1010100039464046D4F81432FFF766FF6889B0F5C8
:10102000017F1DD221464046FFF79AFE284602F076
:1010300092FE012002F0DEFA032000F0E1FB3268AC
:101040000AA180A800F0D6FA80A9012000F022F8B9
:101050000AA1022000F01EF80DF5077DBDE8F0831F
:10106000284602F078FEF7E72800002052656376F4
:1010700020257520627974657300000053746174D3
:10108000653A2050726F672046696E6973686564BF
:1010900000000000012806D0022807D10A460121DD
:1010A000002001F025BA0A460021F9E77047000048
:1010B00010B513A188B0D1E90001CDE9030102F018
:1010C000A3FB02F07DFC00240594069403A807947A
:1010D00000F0AEF90C480D490094CDE9011007ABC2
:1010E00006AA05A90A4802F0A7FC094802F0DCFCA0
:1010F000074801F01BF9064802F0F1FC08B010BDEA
:1011000000000000000200003529000889290008BD
:10111000B400002031B5124C00986168401A41F2C9
:101120008831884203D30098606001F0D9FB0098B1
:10113000E168401AB0F5FA7F03D30098E06000F050
:1011400093FD00982169401A4EF66021884205D32C
:1011500000982061BDE8384000F014BC38BD0000A4
:1011600010000020014801F02FBC0000B400002056
:10117000FEE7704770470000044A0029516901D01A
:10118000014300E0814351617047000000100240BC
:10119000044A0029916A01D0014300E08143916231
:1011A0007047000000100240044A0029D16901D0B4
:1011B000014300E08143D16170470000001002400C
:1011C000044A0029916901D0014300E08143916103
:1011D0007047000000100240F0B52C4A51682C4BBB
:1011E00011F00C014FF00F0504D02A4C042903D054
:1011F000082903D0036028E0046026E051685368A2
:1012000005EA914103F480330D2901D0891C00E0E7
:101210000621BBB1D36A13F4803FD36A03F00F03F6
:1012200003F101030AD0D66AD76AC6F30316761C07
:10123000B4FBF6F4C7F30327BF1C7C43B4FBF3F302
:101240004B43D7E7144B594301605168134C05EAEF
:101250001111635C0168D94041605368072505EAB4
:101260001323E35C21FA03F38360536805EAD32375
:10127000E35CD940C1605268032303EA9232231F22
:101280009A5CB1FBF2F10161F0BD00000010024078
:1012900000127A0040787D0100093D0038000020EE
:1012A0000246002053090949012B0BD0022B0BD019
:1012B000D1F8241002F01F02012393400B4200D00A
:1012C000012070470968F5E7096AF3E7001002405A
:1012D0000149C871704700000010024001490867C9
:1012E0007047000000004242034AD16A21F4704175
:1012F0000143D162704700000010024008B501218F
:101300001020FFF75DFF8020ADF8000010208DF861
:10131000030003208DF8020069460248FFF798FC9D
:1013200008BD0000001001404FF480410148FFF764
:101330000BBD00000018014008B501214120FFF756
:101340003FFF04208DF803000003ADF8000069465C
:101350000148FFF77DFC08BD001801407047000000
:101360000CB500212E4801910091026842F48032B0
:1013700002604FF4A063026802F400320092019A06
:10138000521C0192009A12B9019A9A42F3D1026852
:10139000920342D50121009122490A6842F01002CD
:1013A0000A600A6822F003020A600A6842F0020238
:1013B0000A604168416041684160416841F4A06150
:1013C0004160C16A184A1140C162C16A174A11439B
:1013D000C162016841F08061016001680901FCD5CA
:1013E000416821F47C114160416841F4E811416099
:1013F000016841F08071016001688901FCD5416894
:1014000021F003014160416841F0020141604168FF
:10141000C1F381010229FAD10CBD00910CBD00007D
:10142000001002400020024000F0FEFF44060100D0
:10143000084902780A7042784A7082788A70C278C5
:10144000CA7002790A7142794A7101460020FFF799
:1014500091B900005800002000F0C2B80F480168A0
:1014600041F00101016041680D4A1140416001688D
:101470000C4A11400160016821F48021016041683B
:1014800021F4FE014160016821F0A05101604FF498
:101490007F0181600021C162FFF762BF001002403E
:1014A0000000FFF0FFFFF6FE10B50648064C00787E
:1014B00010B92068FEF712FF2068BDE81040FFF762
:1014C00029BE0000100000200000002000B585B0FB
:1014D00001214FF4E030FFF74FFE01217D20FFF79F
:1014E0006FFEFFF757FBFEF7C1FE02F029F8FFF78A
:1014F0005FFA6846FFF770FE01986421B0FBF1F0D7
:10150000B0F1807F0CD220F07F414FF0E020491EE7
:101510004161044AF02111700021816107210161BC
:1015200005B000BD23ED00E00029018802D041F0A4
:10153000010101E021F0010101807047808C7047BA
:101540008184704730B502881B4B1C4C98420DD0EB
:10155000A0420BD0B0F1804F08D0194DA84205D061
:10156000184DA84202D0184DA84203D122F07005B0
:101570004A882A43154DA84206D0154DA84203D0EB
:1015800022F44075CA882A4302808A8882850A88A4
:10159000028598420AD0A04208D00E4A904205D057
:1015A0000D4A904202D00D4A904201D1097A01863B
:1015B0000121818230BD0000002C01400034014037
:1015C0000004004000080040000C004000100040F3
:1015D0000014004000400140004401400048014028
:1015E000024801680A3101607047000000000020D5
:1015F000FEE700000FB4084B10B504A902AA039837
:1016000000F01CF8044602A9002000F0F3F8204680
:1016100010BC5DF814FB0000F517000802E008C8D4
:10162000121F08C1002AFAD170477047002001E05C
:1016300001C1121F002AFBD1704700002DE9FF4FA6
:101640008BB09A460F4605460026C9E0252837D1BB
:1016500000246D1C6649A04601222B78203B02FA2B
:1016600003F0084202D004436D1CF6E728782E28C8
:1016700017D115F8010F44F004042A280ED06FF09A
:101680002F022878A0F1300109290AD808EB880137
:1016900002EB410100EB01086D1CF2E757F8048BE7
:1016A0006D1C287869283FD006DC002871D063289B
:1016B0000CD0642804D137E0732811D075284ED09F
:1016C00052460D99904706F1010688E017F8040B81
:1016D0008DF8000000208DF80100E946012003E0AC
:1016E00057F8049B4FF0FF3061074FF0000401D41E
:1016F0000AE0641C44450DDA8442FADB19F8041050
:101700000029F6D106E0641C8442FCDB19F80410C1
:101710000029F8D1264404E019F8010B52460D992E
:101720009047641EF8D25AE001CF4FF00A0B002810
:1017300004DAC0F100004FF02D0102E0210504D5CC
:101740002B218DF82410012103E0E10705D0202191
:10175000F7E70DF1200908910CE00021F9E701CF2E
:101760004FF00A0BF9E75946FEF755FD01F130023B
:1017700009F8012D0028F6D1ADEB090000F1200B8E
:10178000600701D44FF00108D84503DDA8EB0B003A
:1017900001E029E000208046002406E009A8524626
:1017A000005D0D999047761C641C08988442F5DB17
:1017B00004E0302052460D999047761CB8F10001A4
:1017C000A8F10108F5DC05E019F8010B52460D9966
:1017D0009047761CBBF10001ABF1010BF4DC6D1CF2
:1017E000287800287FF432AF0FB03046BDE8F08F84
:1017F000092801000A68531C0B6010707047000034
:1018000070B50B4D044601212846FFF78DFE214699
:101810002846FFF795FE03E02846FFF78FFE0446B3
:10182000012CF9D82846BDE870400021FFF77CBEA6
:101830000004004070B5012104468D072846FFF7DB
:1018400073FE21462846FFF77BFE03E02846FFF79C
:1018500075FE0446012CF9D82846BDE870400021E9
:10186000FFF762BE00280BD0026A002A08D0137866
:10187000082B05D10968126B914201D100F034B9EF
:10188000704700002DE9FC41050062D02C6A002C55
:101890005FD0206D4FF03C01471C4FF480364FF66F
:1018A000FF724FF001030AD01E30B0FBF1F0B042DE
:1018B00000D310460004000C208500D12385606D04
:1018C000471C0AD01E30B0FBF1F1B14200D31146E3
:1018D0000804000C608500D1638514F1340000D049
:1018E000606B009070B902F008F9000E7F2802D8F2
:1018F0004FF07F4003E0C0280BD36FF0FF0001F0F2
:1019000058F9009014F1380000D0A06B019010B18C
:101910000BE01148F3E7206B00990840019001208B
:1019200001F047F901990843019004F1300128467C
:1019300002F0CDF86946284602F0CDF801A9284604
:1019400002F0C1F8284602F0CAF80A21204600F049
:10195000E5FCBDE8FC8100000000FFFF70B5046AF3
:1019600005460821204600F0D9FC002204F1300190
:10197000284600F0B7FE6078401C60700120E084CB
:1019800070BD0000164810B5046825E0216A11B347
:10199000488D421E4A85012806D0226A118D481EB4
:1019A000108501290CD016E0216A2046097801290A
:1019B00003D00A2901D005290DD100F09BFA0AE0D5
:1019C000216A20460978012903D00A2901D0052976
:1019D00001D100F0D3FB2468002CD7D110BD00004A
:1019E0007C00002070B506000DD0346A74B100226E
:1019F0004FF49A71104602F084F8E06148B16278C1
:101A000037494AB10BE06FF0090070BD6FF0080074
:101A100070BD4FF0FF3070BD0A68521C0A60096843
:101A200061604168012021620870216A00254870C8
:101A3000216A06208870206AC570606801F0B9F8D4
:101A4000216A4860206A0581206A4581206AC56054
:101A500020780A2803D0052801D0042802D1216A61
:101A60007068C860206A5FF000010561206A456106
:101A7000206A856196F82400884203D9701890F88E
:101A8000250000E0002001F11C02236A491C89B2F4
:101A900098541029EED3002000F12C01226A401C3A
:101AA00080B255544028F7D35FF0000000F16C017C
:101AB000226A401C80B255548028F7D3094801F0AF
:101AC00078F8216AC1F8EC00A5840020226A00F1B0
:101AD000F0015054401C80B24428F7D3002070BD60
:101AE0006400002063538263F8B5046A06460C2143
:101AF000204600F013FC3046FFF774FF05002CD1A0
:101B000001223521204600F093F90421204600F0FF
:101B10009FF904223221204600F08AF9206B01F05F
:101B2000ECFF0146204600F09BF9204600F0CAF980
:101B3000A08CF03081B2E06902F05FF943220A49DB
:101B4000A06802F013FA00964323084AE169A068EE
:101B500002F040FB304600F00BF86078401C6070EB
:101B60001420E0842846F8BD5C4300086043000868
:101B700010B5002809D0046A002C06D0E06908B12D
:101B800002F0E9F80020E061206210BDF8B50546DA
:101B9000046A3348062100682063204600F0BEFB3B
:101BA0002846FFF71FFF06003ED1012235212046BF
:101BB00000F03EF90121204600F04AF902223921C5
:101BC000204600F035F9A98D204600F06AF904227C
:101BD0003721204600F02CF90121204600F038F989
:101BE0000321204600F034F91C21204600F030F992
:101BF0000621204600F02CF9204600F063F9A08C65
:101C0000F03081B2E06902F0F8F843221449A0688C
:101C100002F0ACF900954323124AE169A06802F092
:101C2000D9FA2846FFF7A4FF6078401CC0B2607064
:101C3000062802D20121814000E03C2101EB410055
:101C4000C0EBC1104FF6FF7101EAC00000F2F310C3
:101C50004FF4FA71B0FBF1F0E0843046F8BD0000BB
:101C60005C4300086043000870B50B480025046819
:101C70000EE0206A58B1C18C012903D9A1F10101FC
:101C8000C18404E003D1C584204600F0C0FB246871
:101C9000002CEED170BD00007C00002070B5044621
:101CA0000069002510B101F099FD256160690028E7
:101CB00003D001F093FD6561258370BD0178427802
:101CC000090641EA02418278C07841EA02210843CC
:101CD000704770B54369002473B3068B66B3002266
:101CE00010E0342D03D08D4206D1981870BD921C9F
:101CF00092B29C5C521C04E0521C92B29D5C521C3D
:101D00002A4492B2964202D99D5CFF2DE9D19CB142
:101D1000012C07D00069022C00F12C0006D0C02352
:101D2000002212E000696C308023F9E74023F7E7D6
:101D30008C4202D1104470BD0AE0521C92B2845C05
:101D4000521C224492B29A4202D2845CFF2CEFD100
:101D50000020F0E770B5046A002033216063A063BF
:101D6000E0632046FFF7B5FF18B1801CFFF7A6FF20
:101D7000E0643A212046FFF7ACFF18B1801CFFF762
:101D80009DFF01E0E06C400820653B212046FFF705
:101D9000A0FF18B1801CFFF791FF00E0E06C6065C8
:101DA000206910F1100131D0006920630121204623
:101DB000FFF78FFF28B1801CFFF780FF00F0F9FECE
:101DC000606303212046FFF784FF28B1801CFFF7E2
:101DD00075FF00F0EEFEA0631C212046FFF779FF9F
:101DE00028B1801CFFF76AFF00F0E3FEE0630621E4
:101DF0002046FFF76EFF060019D070788008206437
:101E0000022801D90220206400250DE00020CCE743
:101E100006EB8500801CFFF751FF00F0CAFE04EBC3
:101E200085016D1CEDB24864206CA842F0D870BDED
:101E300010B5838C046A1C445B1C838484F8F01006
:101E4000818C036A0B44491C818483F8F02010BD07
:101E5000828C036A1344521C828483F8F01070470A
:101E600010B5828C046A0B0E1444521C828484F8D0
:101E7000F030828C046A0B0C1444521C828484F867
:101E8000F030828C046A0B0A1444521C828484F859
:101E9000F030828C036A1344521C828483F8F01061
:101EA00010BD10B5828C046A0B0A1444521C828443
:101EB00084F8F030828C036A1344521C828483F8C5
:101EC000F01010BD002814D0818C036AFF220B444F
:101ED000491C818483F8F020002205E0036A0B444A
:101EE000491C818483F8F020818C4429F6D38B0728
:101EF000F4D17047F8B5046A05460421204600F085
:101F00000DFA2846FFF76EFD060029D10122352182
:101F10002046FFF78DFF03212046FFF799FF02229D
:101F200039212046FFF784FFA98D2046FFF7B9FF2E
:101F30002046FFF7C7FFA08CF03081B2E06901F0C6
:101F40005CFF43221149A06802F010F8009543237A
:101F50000F4AE169A06802F03DF92846FFF708FE44
:101F60006078401CC0B260700A2803D24FF47A71C6
:101F7000484301E042F2107080B200F2F3104FF4D7
:101F8000FA71B0FBF1F0E0843046F8BD5C43000824
:101F9000604300082DE9F041046A51680546E2609B
:101FA00008780026904602287AD1002095F824204F
:101FB00008E02B180F1893F825303F7FBB426FD1F4
:101FC000401CC0B28242F4D8486801F096FD6168B6
:101FD000884265D1204600F054FA002860D13521AE
:101FE0002046FFF776FE00285AD08078052804D0D6
:101FF000062819D0022839D052E02078012806D0CE
:1020000003280CD004280AD0052808D048E0284628
:10201000FFF7A0FEE6842846FFF7A0FC40E0E68438
:102020002846FFF72FFC3BE02078032805D0012845
:1020300003D0042801D0052832D1E68428462F6A2F
:1020400001F038FD1C49284601F041FD1A49284697
:1020500001F039FD1849284601F03DFD0C213846B4
:1020600000F05CF92846FFF791FD19E0207806287A
:1020700016D1E6842F462D6A36212846FFF729FE21
:1020800070B1801CFFF71AFE00F093FDE86228692A
:1020900010F110010DD000692863384600F0BCF83B
:1020A0002046FFF7FBFD404601F055FEE660BDE827
:1020B000F0810020F0E700005C430008F8B5046AF6
:1020C00005460D21204600F029F90020E0626063FA
:1020D0002063E063A06360652065E06420642846B7
:1020E000FFF780FC060022D1012235212046FFF7B0
:1020F0009FFE07212046FFF7ABFE2046FFF7E2FEDA
:10210000A08CF03081B2E06901F077FE04F12C017F
:1021100043220F46A06801F029FF009543233A4669
:10212000E169A06802F056F82846FFF721FD6078C3
:10213000401CC0B260700A2803D24FF47A71484341
:1021400001E042F2107080B200F2F3104FF4FA7125
:10215000B0FBF1F0E084284601F0ACFC06492846CB
:1021600001F0B5FC0449284601F0ADFC02492846BF
:1021700001F0B1FC3046F8BD5C430008F8B5046AD4
:1021800005460521204600F0C9F82846FFF72AFC3D
:1021900006002BD1012235212046FFF749FE0321FD
:1021A0002046FFF755FE022239212046FFF740FE68
:1021B000A98D2046FFF775FE2046FFF783FEA08C11
:1021C000F03081B2E06901F018FE04F12C014322E5
:1021D0000F46A06801F0CAFE009543233A46E16924
:1021E000A06801F0F7FF2846FFF7C2FC6078401CAA
:1021F000C0B260700A2803D24FF4FA61484301E08C
:1022000044F6206080B200F2F3104FF4FA71B0FB94
:10221000F1F0E0843046F8BDF8B5046A05460121C6
:10222000204600F07BF82846FFF7DCFB060056D17D
:10223000012235212046FFF7FBFD03212046FFF751
:1022400007FE022239212046FFF7F2FDA98D204624
:10225000FFF727FE042232212046FFF7E9FD206B1D
:1022600001F04BFC01462046FFF7FAFD042236211F
:102270002046FFF7DDFDE06A01F03FFC0146204605
:10228000FFF7EEFD042237212046FFF7D1FD0121A3
:102290002046FFF7DDFD03212046FFF7D9FD1C2175
:1022A0002046FFF7D5FD06212046FFF7D1FD204649
:1022B000FFF708FEA08CF03081B2E06901F09DFDCF
:1022C00000954323134AE169A06801F083FF43228C
:1022D0001149A06801F04AFE2846FFF749FC6078E2
:1022E000401CC0B26070062802D20121814000E08B
:1022F0003C2101EB4100C0EBC1104FF6FF7101EA38
:10230000C00000F2F3104FF4FA71B0FBF1F0E0847A
:102310003046F8BD604300085C43000802788A42FA
:1023200002D00170002141707047000070B50500B7
:1023300034D095F82E002C6A20F0080085F82E0085
:10234000A88D4FF0FF36B0F5107F25D34CB3A068B1
:1023500008B101F015FFE06808B101F0FCFC58215C
:102360002046FDF73AFF01F0FBFEA06000B34422D7
:10237000154901F0CDFD43221349A06801F0F6FD97
:102380002A461249A06801F0F8FE2846FFF7FEFB36
:10239000A0B1284600F01CF8304670BD6FF009006F
:1023A00070BD582001F04AFA0400F5D02C62D6E73F
:1023B000204601F013FA00202862EDE715F82E1FE1
:1023C00041F00801297070BD5C430008951F0008AA
:1023D00070B5046A050019D095F82E00002C20F085
:1023E000080085F82E0011D0A068002610B101F079
:1023F000C7FEA660E06810B101F0ADFCE6602046C3
:10240000FFF74CFC204601F0E9F92E6270BD10B5D3
:10241000026A044611780C2911D006290FD001292F
:1024200011D0082917D0052921D0042928D15078A6
:10243000082820D82046BDE81040FFF75BBDBDE866
:102440001040FFF7A3BB5078052814D82046BDE8FC
:102450001040FFF7E1BE50780128204603D8BDE8C0
:102460001040FFF77BBABDE81040FFF70BBABDE89C
:102470001040FFF783BE2046FFF720FE2046DEE730
:1024800010BD70B5040025D0E06830B32046FFF7DA
:1024900005FCE0684FF0FF350089F02806D9F038D8
:1024A00080B2208301F0CAF96061C8B1F02001F068
:1024B000C5F92061010015D00023F022E06801F089
:1024C00016FC616921B1228BF023E06801F00FFC5A
:1024D000002070BD6FF0090070BD6FF0080070BD86
:1024E000284670BD606901F079F900206061F7E766
:1024F0002DE9F04190460446002501F0010611E067
:1025000018F8057004F01F000EB140F0400040F0D4
:10251000800001F06FF8384601F096F86D1C641CDD
:10252000EDB2E4B24046FDF76FFEA842E8D8BDE840
:10253000F0812DE9F84390460E46050060D0B8F8CA
:102540000A002A2859D30120D8F8044000F033FBB0
:10255000E189884251D140F2046000F02CFB618A8D
:1025600088424AD14FF4006000F025FB218A88425E
:1025700043D140F6060000F01EFBA18988423CD101
:10258000E0690090D4F82610686820B1814202D139
:1025900001273B4601E000273B4604F1160269464D
:1025A000284601F06FFEA08A00F005FB012802D04A
:1025B000022822D11DE007B3022000F0FCFAA0821D
:1025C000E069C4F826006868E0610622521E12F035
:1025D000FF0204EB0200817D80F82010A154B15C61
:1025E0008175B15C8171F1D1AA6941462846904755
:1025F00003E069462846FFF735F9404601F0ABFB9A
:10260000BDE8F88330B400280ED049688268446879
:10261000D1F81A3014401340A34205D100238A1D7B
:1026200030BC1A3101F02EBE30BC70472DE9FC41A0
:102630000E46054614460E21304601F0AEFB18B199
:102640006FF00100BDE8FC812946204600F0A4FBA4
:1026500008B1234B28E04FF0704001F04EFA21689A
:1026600000EA01074FF0604001F047FA874222D1AB
:1026700001208DF8000000208DF801005E208DF80B
:102680000200206801F039FAC0F306408DF803001B
:10269000206801F032FA000A8DF80400206801F089
:1026A0002CFA8DF805006B4605F1250231462846C7
:1026B00000F0FAF8C6E7A86821686A68014002409D
:1026C000914203D0E86838B105F10C043246214646
:1026D000284600F007F8B5E76FF00300B2E7000006
:1026E000644300082DE9F05F0D46824600F1250B9A
:1026F00014464FF0FF385146284600F04DFB08BB0A
:102700004FF0704001F0F9F9296800EA01064FF036
:10271000604001F0F2F9864214D09DB1286888B17A
:102720000121284600F08CF900280DDBDFF8B0907D
:1027300000EB800609EB8607B87B38B1012807D08B
:1027400034B10BE06FF00900BDE8F09F0120B873D1
:102750002946504600F096F8804604B3B87B4D46B3
:10276000022802D0012808D038E007F108035A46B1
:102770002146504600F098F82FE02046017B0129C1
:102780000ED001890022032001F0BBF9070025D0FB
:10279000214601F064FA58B1384601F0DCFA1DE038
:1027A00000680028EAD12746204601F04DFBAFB172
:1027B000032001F031F90100EED00020C1E900074B
:1027C00055F8260008B905E010460268002AFBD13A
:1027D000016001E045F82610002080464046B3E73E
:1027E000B87900202DE9F05F1746DDE90B9B88469C
:1027F00082461E4600222A21032001F082F90500AC
:102800003CD06C680D9800F0D6F9A0820620401EDE
:1028100010F0FF0004EB0001325C8A7519F800200B
:1028200081F820203A5C225418F800208A71EED1F9
:102830000A980068E061DBF80000C4F82600012077
:1028400000F0B9F9E0814FF4006000F0B4F92082A3
:1028500040F2046000F0AFF9608240F6060000F03C
:10286000AAF9A081DAF81820504629469047044674
:10287000284601F070FA2046BDE8F09F4FF0FF3087
:10288000FAE700001FB50123064C021DCDE9021333
:10289000CDE9002400F125031946A21FFFF7A2FF8E
:1028A00004B010BD6A4300082DE9F0414D680E46A2
:1028B00007460624641E14F0FF0405EB0401185DAE
:1028C0002855105D8871F5D14FF4006000F073F960
:1028D000A88131463846BA69BDE8F041104700008A
:1028E0002DE9F0410025124CA84600BF05EB8507F5
:1028F00004EB8706F07B401CC0B2F073B17B022969
:1029000002D0012903D00DE0F02802D20AE002280B
:1029100008D354F8270018B100F03CF944F8278098
:1029200086F80E806D1CEDB20A2DDFD3BDE8F08174
:10293000B879002070B5044640680D46808900F0E3
:102940003AF9B0F5006F04D0A0F5006006380AD15E
:1029500012E021462846FFF755FE6FF00D01204694
:1029600001F01BFA18B1204601F0F5F90AE02946FA
:10297000204600F0BFFA05E0224605F12501284671
:10298000FFF7D7FD002070BD10B50446082000F009
:1029900055FF90B17321E06184F82F10742184F801
:1029A0003010074961610749A16104F12501016007
:1029B000204600F073FE002010BD4FF0FF3010BD28
:1029C0002D2600080D3700082DE9FE43814600261C
:1029D0006846FDF725FFDDE901710098884681B260
:1029E0000322104601F08DF805000AD00446B919FB
:1029F00062896068FDF7D8FB608924680644002C72
:102A0000F5D10E484FF00041C8F8001041690906A1
:102A100003D5802141610021816065B1D9F8102082
:102A2000494628469047040002D0284601F093F911
:102A30002046BDE8FE834FF0FF30FAE700900240E9
:102A40002DE9F35F4FF00A0A4FF00001DFF83CB1C7
:102A50000400D14652460D460E4657460B4616D048
:102A60004B4890F8008008EB880C0BEB8C0090F83A
:102A70000EC0BCF1020F0AD1D4F800C040688445F2
:102A800005D14FFA88F0BDE8FC9F0A2A07D1DFF88C
:102A9000FCE001EB810C0EEB8C00807B60B101EB64
:102AA000810B0EEB8B0090F80EC0BCF1010F05D02E
:102AB000BCF1020F1AD02AE04AB228E02CB1D4F8B7
:102AC00000C0D0F80480C44517D05EF82BC0C07B8E
:102AD000BCF1000F04D0984219D34FB2034616E060
:102AE000A84214D34FFA81FA054610E04CB1D4F84D
:102AF00000C0D0F80480C44503D12548017048B215
:102B0000C1E7C07BB04202D34FFA81F90646491CA7
:102B1000C9B20A29B9D301994FF0FF304FF000082C
:102B20000A2A05D08907AED40A2A06DAD5B21CE0F3
:102B3000C907A8D001998907A5D4B9F10A0F02DA0B
:102B400009F0FF0511E0BAF10A0F02DA0AF0FF05F9
:102B50000BE00A2F97DAFDB20C4E05EB850756F80D
:102B6000270000F017F846F82780084805EB850293
:102B700000EB8200414680F80E800CB12268426072
:102B8000C1730348057068B27DE70000B879002082
:102B90009C00002070B5044608E02546D5E90040B9
:102BA00001F0D9F82946032000F0FEFE002CF4D1F4
:102BB00070BD00BA704740BA70470A46032100F062
:102BC0008AB82DE9FE4F446805468A46208800F001
:102BD00096FFC0F303204FEA8009C9F1000188463F
:102BE000284601F0DAF8002870D1288904286DD32E
:102BF00068680078082869D101264FF0704000F01D
:102C00007CFF216900EA01074FF0604000F075FF8A
:102C1000874200D10026514604F1100000F0BCF8B4
:102C2000002853D1002E51D0288908284ED3284699
:102C300000F08EF8E8BB2221284601F0AEF8D0B1B2
:102C40004946284601F0A9F898BB298900220220AC
:102C500000F057FF060039D0294601F000F840BBCC
:102C600041463046746801F098F810BB284601F0E0
:102C700072F8354605E06FF02101284601F08DF825
:102C8000B8B96868E1682269E260216100260670CF
:102C90004680208900F033FFC0B240F47F40FFF748
:102CA0008AFF208166814946284601F076F800B9FE
:102CB00000E00BE00121CDE90061FF230022CDF807
:102CC00008A004F10C01284600F0EAF92846BDE806
:102CD000FE4F01F040B82DE9FC4791460E46804674
:102CE00000222421012000F00CFF050024D06C6894
:102CF000D8F804701C22267084F801900026A68063
:102D0000E6806868D8F804100830FDF74DFA668050
:102D10006989204600F016F860800120CDE9006046
:102D2000FF2307F10C020021284600F09FF92846F6
:102D3000BDE8FC4701F00FB8BDE8FC870A460B214F
:102D4000FFF7C9BF10B500F0F7FCC04380B210BD5B
:102D500070B500242646054613E06989686800F0CE
:102D6000EBFC204481B201EB1044A87AC00707D0E5
:102D7000C6F10100C6B2E0B2C4F3072141EA002463
:102D80002D68002DE9D126B1E0B2C4F3072141EA54
:102D90000024E04380B270BD0068421C12D088B1AC
:102DA00091F82E2092070BD54A68824208D0896894
:102DB00000EA01030A40934202D10143491C01D0B9
:102DC00000207047012070472DE9F74F84B00222A0
:102DD00005984FF014080021858D104600F091FEF3
:102DE000070020D042487D813D8120F003047C60B3
:102DF0000498142241682046FDF7D6F9E08800F0D7
:102E00007EFEC0F30C0900F4005002900498008983
:102E1000143886B2143DE81705EB5070C0F3CF00AC
:102E2000CDE9000553E04FF0FF3007B0BDE8F08F6B
:102E30000198864201DC012000E000205FEA000AE0
:102E40000298C9F30C0545EA000547D0304680B228
:102E500083460246434604F11401049800F047FFFC
:102E600040441FFA80F82846FFF7A5FEE0800BF1EA
:102E7000140080B2FFF79FFE608000206081142163
:102E80002046FFF75FFF6081BAF1000F05D006F121
:102E9000140081B2384600F0B0FF00221146022033
:102EA00000F02FFE05001ED0394600F0C6FE059842
:102EB0002946069A43699847284600F04CFFA6EB3E
:102EC0000B00009986B209EB01001FFA80F9002E71
:102ED000AED1384600F03FFF0020A6E7009845F449
:102EE0000055C000B3E7384600F035FF9BE700000F
:102EF000DA7300202DE9F05F446806468846208892
:102F000000F0FDFD0421B1EB103F12D1208800F04C
:102F1000F6FDC0F303204FF6FF7101EA80096088D7
:102F200000F0EDFD728901464A4502D3308988429E
:102F300003D2304600F00FFF60E0304600F05DFF46
:102F4000DFF820A10127454604F1100B284600F0C8
:102F500097FD68B1281D0BD0686848B1216981428E
:102F600004D029465846FFF717FF08B15DB117E0B6
:102F70001FB10027DAF8005000E02D68454500D168
:102F80002D68002DE2D1208900F0B9FDC0B21128D2
:102F900006D104EB0900408800F0B1FD44282BD095
:102FA000414604F10C00FFF7F7FE0028C1D14FF0B5
:102FB000704000F0A2FDE16800EA01074FF06040B8
:102FC00000F09BFD8742B4D0002DB2D043F6FF70D5
:102FD000FFF7F1FDE188084205D0304600F0C6F861
:102FE00006000BD07468204D41463046C5E9018487
:102FF00000F05AFF28B131E04546E5E70020BDE882
:10300000F09F208900F07BFDC0B201280CD0112870
:10301000414605D004F11000FFF7BEFE48B11AE0AA
:10302000304600F0D5FF19E041463046FFF7C9FDB4
:1030300014E04FF0704000F060FD216900EA0107E4
:103040004FF0604000F059FD874204D00221304625
:103050007460FFF7B2FD304600F07DFE002068602E
:10306000A860CBE77C000020880000202DE9FE430B
:103070008146DDE90A541F4616468846104600F090
:103080003BFA50B10095CDE901403B4632464146FE
:10309000484600F005F8BDE8FE836FF00300FAE74C
:1030A0002DE9F05F1F46DDE90BA5DDF828B05FEAEA
:1030B00002088946064641D01421304600F06DFED4
:1030C00018B16FF00100BDE8F09F7468208900F02E
:1030D00016FD67F31F20FFF76EFD208100F00FFD46
:1030E00020F0FF0040EA0A00FFF765FD2081D8F8D4
:1030F000000020611FFA8BF040F48A40FFF75BFD6F
:1031000020803089FFF757FD174F60804FF0000A8D
:10311000A4F806A03888FFF74EFDA0803888401C30
:103120003880B9F1000F02D0D9F8000010B9281D7D
:1031300000D06868E060A4F80AA002E0706800F1BE
:103140001008A88D48B13189814206D942462946E6
:103150003046BDE8F05FFFF737BE424631462846AD
:103160006B69BDE8F05F1847880000202DE9F14F3A
:103170004FF0000A00984568288800F0C0FCC0F3B2
:10318000032005287ED1E88800F0B9FCC0044FEA8E
:103190001049688800F0B3FC0446288800F0AFFCB2
:1031A000C0F30320404204EB80001FFA80F800982F
:1031B00000F04CFD514E0746308838440A2809D9A2
:1031C0003946284600F062F900285BD03088384440
:1031D0000A2857D84FF0000B74680DE06069E96861
:1031E000884207D1A0692969884203D1A089A988AA
:1031F000884204D0A2462468002CEFD106E02CB10E
:10320000E88800F07CFCC00419D023E0022000F024
:1032100003FC04000AD13946284600F037F9B842C9
:1032200066DB022000F0F8FB040061D02021FCF7EF
:10323000D4FF0320E07770682060746004E0E089C8
:1032400000F05DFCC00405D01422294604F10800FA
:10325000FCF7AAFF308838443080E88800F04FFC43
:10326000800406D4A07F40F00100A07709EB08009D
:10327000A0832046009900F043F8002836D0A08BA8
:10328000143000E034E0A0836068142204F10801E7
:10329000456828462F68FCF787FFA08BFFF78BFC5B
:1032A0006880A5F806B0A5F80AB014212846FFF7F3
:1032B00049FD68816FF01309D4F8048009E049469C
:1032C00038467D6800F069FD3946404600F0A1FCB3
:1032D0002F68002FF3D15146204600F08DF840466C
:1032E00000F0B4FC3188081A30804046BDE8F88F01
:1032F000009800F030FD0020F8E700009400002066
:103300002DE9F047D1F8049006460D4600244FF011
:103310000108B9F8020000F0F2FB0746B9F8000016
:1033200000F0EDFBC0F30320404207EB8007B9F843
:10333000060000F0E4FBC004010C68680022026093
:10334000CA19818097B2C78073681EE05A68B2F8C4
:1033500004C061450DD2036044B1B4F806C06145B4
:103360003CD391888F4239D8256000E0756073B1F5
:103370001AE033D0D388994230D324B1E38863452F
:1033800001D04FF0000813681446002BDED154B171
:103390002560E1888288914206D0B17F4FF0000815
:1033A000C90714D118E07560B17FC90714D0B8F10E
:1033B000000F0CD071684968898831B9016831B152
:1033C0004968C0888A88904204D04FF0000840467F
:1033D000BDE8F0870846F1E70020F9E7284600F04D
:1033E00035FC014603480288511A0180284600F046
:1033F000B2FCF1E794000020074B30B40A465C6849
:103400000168844201D1596000E01160014630BC7E
:10341000022000F0C9BA0000940000202DE9F0411C
:1034200044680646884660680025818891B900682E
:103430007060142206F108016068FCF7B5FE0121F6
:103440002046FFF77BFC204600F000FC05462046A6
:1034500000F081FC746809E060682746046838461B
:1034600000F0F4FB0544384600F075FC002CF3D165
:1034700041463046FFF7C0FF03480188491B0180E1
:103480002846BDE8F0810000940000202DE9F041BD
:10349000184F8846064600240022114615467868D3
:1034A0001AE04369D6F80CC0634509D18369D6F8A0
:1034B00010C0634504D18389B6F804C0634507D0C2
:1034C0006D1C22B1C37F92F81FC0634500D802462D
:1034D000036803B1014618460028E2D11AB110462C
:1034E000FFF79CFF0444444501DA012DD4DC20465B
:1034F000BDE8F0819400002070B505460E480468D0
:103500000DE0204600F0BCFA40B1A068296862686E
:1035100001400240914201D1204670BD2468002C38
:10352000EFD1064C206820B100F0AAFA08B120685B
:1035300070BD002070BD00007C00002080000020D5
:10354000F8B54EF2FF00ADF8000010248DF80340EE
:1035500003258DF8025069462348FDF779FB0120C9
:10356000ADF80000214E8DF803408DF802506946F9
:103570003046FDF76DFB382000F03CF80520FEF7E3
:103580003FF9382000F036F80520FEF739F93820E9
:1035900000F030F80520FEF733F9082000F02AF893
:1035A0000520FEF72DF9012000F024F80520FEF794
:1035B00027F9062000F01EF80520FEF721F9482023
:1035C00000F018F80A4D0024285D00F03DF8641C56
:1035D000E4B2182CF8D30C2000F00CF83046BDE80B
:1035E000F8400121FDF7B9BB00140140001801406B
:1035F0002C43000870B5134D04464FF40051284683
:10360000FDF7A9FB4FF480412846FDF7A4FBFF21FD
:103610002846FDF7A0FB21462846FDF79EFB4FF408
:10362000004421462846FDF798FB6420FEF702F986
:1036300021462846FDF78FFBBDE870400A20FEF7C3
:10364000F9B800000014014070B5134D04464FF462
:1036500000512846FDF781FB4FF480412846FDF7D5
:103660007AFBFF212846FDF776FB21462846FDF729
:1036700074FB4FF4004421462846FDF76EFB64209E
:10368000FEF7D8F821462846FDF765FBBDE87040F7
:103690000A20FEF7CFB800000014014070B50621E3
:1036A00000F8241F16490A7842704A7882708A7896
:1036B000C270CA7802710A7942714979817140F207
:1036C000DC5101813221817204220E490E48FCF73F
:1036D000E5FE0D4906224031A1F1A000FCF7AAFE4B
:1036E000094D00244FF4400605EB04103146FCF769
:1036F000F9FE641C042CF7DBBDE87040FDF7C0B890
:1037000058000020282500204801002070B5002521
:10371000FCF70AFF06460C4607E0628970196168EB
:10372000FCF742FD608924680544002CF5D1A8B25D
:10373000FDF7F6F8002070BD30B4002207E00378F2
:103740001C024378801C2343891E1A4489B2012934
:10375000F5D811B1007802EB002290B200EB1240D4
:10376000010C02D081B201EB104030BC80B2FFF7F7
:1037700022BA000010B5FDF7DFFDFDF7D5FDB8B1A9
:1037800012480168124A1140B1F1005F05D0FDF7FF
:10379000B5FD104980200861FEE741680E4CE160EC
:1037A000A1600068FCF7E7FCA0688047002010BD1E
:1037B000FDF78CFEFDF77CFCFDF7C0FBFCF7BAFEC5
:1037C00008B1FDF7CFFCFDF76FFEF7E700900008AA
:1037D0000000FE2F001001400000002000280FD044
:1037E00008494A6890420BD38A68904208D2083848
:1037F00000220271CA68904200D2C86000F02ABB61
:10380000704700006800002010B50A480A4A20F0FE
:1038100003004FF480535060002103804180017108
:1038200000F58051012491600C710B804B80147065
:10383000D06010BDEB3C002068000020F0B50028EF
:1038400047D0C01C4FF6FC7100EA01044FF4805CC5
:103850000C2C01D20C2401E064453FD8204AC4F569
:103860008055D6685368F01A81B235E05818077948
:1038700087BB07887F1A083FA7422CD3058804F12D
:10388000140E6D1A083D0127754514D30C440834F5
:10389000A5B25C194FF0000E84F804E0B0F800E027
:1038A000A4F800E06180058007712188614503D09C
:1038B0009C1C0D5300E00771B04209D1D2E90241CE
:1038C0000D792DB1A14203D009881944D160F7E7E1
:1038D0000830F0BDFFE7595A8D42C7DC0020F8E7F9
:1038E000680000202DE9F04FC91C4FF6FC72114012
:1038F0004FF480590C2901D20C2101E0494510D820
:10390000284D6C68A0420ED3AA6890420BD2A0F159
:103910000802131B17889BB2FE1A083EB6B2B142CA
:1039200003D94FF00000BDE8F08FFCD0AA461D4D32
:1039300007EB040C4FF0000BEF689CF804806D68F7
:10394000B8F1000F05F1020516D001F1140CB445D1
:10395000E9D8194408318EB2A119B94201D2CAF886
:103960000C1081F804B014880C804B8016800988F4
:103970004945D8D04E53D6E719440831BCF8006009
:1039800089B2674502D16718CAF80C700C4484F8F4
:1039900004B026806380118022884A45C3D05153E9
:1039A000C1E7000068000020002905D0034A52F852
:1039B00020300B6042F8201070470000FC4C0020C3
:1039C000F0B50020401C80B20628FBD31048104BF5
:1039D00020F0030200200F4D07461B3B05F10C04AD
:1039E00043F82070002109E053F82060166043F886
:1039F000202035F81060491C324489B234F8106038
:103A00008E42F1D8401C80B20628E9D3F0BD0000F8
:103A1000174D0020444300080146062801D300202A
:103A20007047044A52F821000028F9D0036842F890
:103A300021307047FC4C00202DE9F041044606A8D7
:103A4000E0C800206060A060E06084F82E00C4E957
:103A500007500A4D287884F83100401C2870204611
:103A6000276100F012F82046B04710B10020BDE8F1
:103A7000F0816868206020466C60F8E778000020DC
:103A800090F82E0000F00100704710B5044600F0D9
:103A90001EF81146204600F01EF82046BDE81040F2
:103AA000194600F010B80000014988607047000016
:103AB0007800002090F82E10CA0703D021F00101F1
:103AC00080F82E10704701B10968C160704701B1DC
:103AD00009684160704701B109688160704790F8DA
:103AE0002E10CA0708D141F0010180F82E10890676
:103AF00002D5011DFEF7C6BE704700BA704740BA36
:103B000070472DE9F05F16460D46002730B10128B9
:103B100005D0022804D003284DD102E01427143721
:103B20000E374FF0010A4FF00008F6B3012E5ED0B9
:103B3000022E5CD0032E3ED10520FFF76DFF04005E
:103B40003AD0E0191330267320F00300C4E9008056
:103B5000FF1C27F00300C0F5BE6041462581A84246
:103B600000DD284660815746A4F80EA0A1462D1A14
:103B70004FF4BE6B884616E00520FFF74DFFB8B145
:103B8000067380F80D80C0F80080A9B2C9F8000063
:103B90000181594500D35946418100F1100242602C
:103BA000C7816D1A8146002D00E007E0E4DC2AE0C1
:103BB000204600F0D0F80020BDE8F09F07F1130088
:103BC00020F00301E81C20F00300084480B2FFF756
:103BD00035FE0400F0D0E019133020F003006060DF
:103BE00025816581C4F8008084F80C800BE00420F6
:103BF000FFF712FF0400DFD0C4F80480258165813F
:103C0000C4F800802673A4F80EA084F80D80204626
:103C1000D2E710B500280FD000290DD004E00389A9
:103C20000C892344038110460268002AF7D10289D7
:103C30000B891A440281016010BD10B50C46FFF7D4
:103C4000E8FF2046BDE8104000F0FEB8002102E089
:103C5000491C0068C9B20028FAD1084670472DE90E
:103C6000F0474FF000070C4605003E4604D01CB15B
:103C700028892189884203D26FF00900BDE8F087C6
:103C80006FF0080968896189C01B891B884201DBC4
:103C900088B200E080B28046606842468119686858
:103CA0003844FCF781FA07EB080087B206EB0800FE
:103CB00086B26889B84201D12D6800276089B04278
:103CC00001D8246800262CB160892189884201D15D
:103CD000206830B93DB168892989884203D12868B4
:103CE00008B14846CAE7002CCCD10020C6E72DE930
:103CF000F047164689464FF00008002806D0B9F173
:103D0000000F02D00027044620E00020BDE8F08725
:103D10002BB16089984202D8181A83B215E06089E5
:103D2000C01A85B2B54200D9354660682A46C11826
:103D300009EB0700FCF738FA08EB05001FFA80F8DA
:103D4000781987B2701B86B2002324680EB1002C4C
:103D5000DED14046DAE770B5002815D00024C189CD
:103D6000491E0904090CC1810DD1017B0568032995
:103D70000BD001290CD002290AD0FFF72FFD641CBB
:103D8000E4B22800EBD1204670BD0146052001E0D9
:103D900001460420FFF708FEF1E710B541B138B144
:103DA000002907DA4A4293B242899A4223D302E0B9
:103DB000002010BD8BB2027B446832B1032A04D0CC
:103DC000022A0AD0012A08D015E0621A00F1100375
:103DD00042609A4208D244600DE000290BDA428921
:103DE0009A4208D3621A426042890A444281028997
:103DF00011440181DCE7012010BD70B502898A42BF
:103E000021D98A1A0D46044605E0281A85B2208970
:103E10001044208124686089A842F6D3207B50B9E1
:103E20006089A84207D0A088001B284481B22046A0
:103E3000FFF758FD044665812581206808B1FFF72A
:103E40008AFF0020206070BD002802D0C189491C73
:103E5000C181704730B5134903884A681344941CE4
:103E600098420DD01D795DB98D68AB4208D0CD6800
:103E70009D4200D1C8601D8805801B88851A1D538E
:103E80004388134483420BD01D79002D08D1CD689F
:103E9000854200D1CB60018819800088991A0153AE
:103EA00030BD0000680000202DE9F04746688246DA
:103EB00000273089FFF723FEDFF8509000F0FF085D
:103EC0000025D9F800401CE0217C414516D1D4F8EA
:103ED00014C0BCF1000F11D006F10C03524621466C
:103EE000A069E04750B14FF0000A012735B1E06802
:103EF000E860D9F80010E160C9F800402546E468A0
:103F00000FB9002CE0D13846BDE8F08784000020CE
:103F1000F0B5154B00251C6803E0A04200D1012537
:103F2000E468002CF9D101B109680160A2B91968EF
:103F30004FF480520C4647F6FF7607E04F8A9742CF
:103F400003D1521C92B2214600E0C96821B1B242AD
:103F5000F4D16FF00A00F0BD428215B91968C16052
:103F600018600020F0BD00006000002070B516460B
:103F7000428A0D46044622B90146FFF7C9FF0028D0
:103F800010D155B128686060A682207C094A40F0B3
:103F9000040020741068014606E00020F3E7844224
:103FA00001D1002070BDC0680028F8D1E160146024
:103FB000F7E7000060000020044909684160002123
:103FC0008182017C21F00401017470475C43000888
:103FD0002DE9F84F4568064689462888FFF78FFD8A
:103FE000C0F303214FF0080B30890BEB81018142B4
:103FF00069D82888FFF783FDC0F303208000414281
:104000003046FFF7CAFE00285DD1494605F1100091
:104010007468FEF7C1FE00902088FFF770FD074628
:104020006088FFF76CFD00240246442807D0DFF8C3
:104030002CA100200146DAF800301C464EE0432F48
:1040400050D1D9F82000E8B38068D8B3011D04D05E
:10405000416811B1EA68914244D1044647E000BF8B
:10406000B4F812C0944537D1DDF800C0BCF1000FA0
:1040700005D17CB1D4F800C0BCF1000F0AD0D4F84F
:1040800000C0D5F81080C44504D0DDF800C0BCF1F4
:10409000000F21D029B994F810C05FEA4C7C00D4FD
:1040A0002146B4F814C0BC4516D114F1040C08D054
:1040B000D4F804C0BCF1000F03D0D5F80C80C4457F
:1040C0000AD101E00EE044E020B1E268C260E360A2
:1040D000CAF8004024B10AE02046E468002CBFD1B1
:1040E0000C0004D1D9F804002969884231D16FF05D
:1040F00007013046FFF751FE58BB6CB1D4F818C029
:10410000BCF1000F25D0009705F10C033246214683
:10411000E069E047BDE8F88F0098D0B94FF07040F3
:10412000FFF7EBFC296900EA01044FF06040FFF75C
:10413000E4FC84420DD02888FFF7E1FCC0F30321A2
:104140000BEB81013046FFF728FE03213046FEF7D6
:1041500034FD3046BDE8F84FFFF7FDBD600000209C
:1041600010B50120FFF758FC040004D02021FCF713
:1041700034F8FF20E072204610BDC0E906127047F7
:1041800009490A68824209D1D2680A6008E0D16808
:1041900019B1814201D1C168D1600A46002AF6D125
:1041A00001460120FFF700BC60000020F8B507467B
:1041B0001D460E4614461046FFF79EF938B1009092
:1041C0002B4622463146384600F004F8F8BD6FF021
:1041D0000300F8BD2DE9FE4F9246428ADDF830908B
:1041E0001E468846044622B90146FFF791FE002884
:1041F00011D108214046FFF7D0FD70B100220821FF
:104200000120FFF77EFC050003D04146FFF715FDB6
:1042100004E04FF0FF30BDE8FE8F4546608A6F68CE
:10422000FEF7C9FC38803046FEF7C5FC78800020D8
:10423000F8806CB1206858B1D9F8041088420AD0CF
:10424000454502D02846FFF786FD6FF00800E2E7FB
:1042500009F1040600E026462889FEF7ACFCB88088
:10426000A17A11228DE80602E37A524631462846A9
:10427000FEF716FF0446454502D02846FFF76BFDC2
:104280002046C8E72DE9F047984616460D0004463B
:1042900013D0286888B121462846FEF77DFD60B915
:1042A0004FF07040FFF729FC296800EA01074FF042
:1042B0006040FFF722FC874203D16FF00900BDE8A0
:1042C000F08741462846FEF7BBFB0028F7DB164A7D
:1042D00000EB8005022302EB850106208B730C6145
:1042E000401E10F0FF0001EB0007335C3B72F7D17A
:1042F000C87304F1250990460FE00A6848F82520A4
:1043000003204F68FFF750FB33464A4639462046A4
:10431000FEF7CAFA3846FFF71EFD58F825100029A7
:10432000EBD10020CBE70000B879002001030D0D90
:104330000D0301000810001C00100800070507000D
:10434000000000001C0020002000080010000006F3
:104350000400050005001E00020006000000000029
:10436000FFFFFFFFFFFFFFFFFFFF00000000000057
:104370009043000800000020B40000001C16000854
:1043800044440008B4000020CC7D00002C16000836
:10439000000000000000000000000000000000001D
:1043A000000000000000000000000000000000000D
:1043B00000000000000000000000000000000000FD
:1043C00000000000020406080000000001020304CF
:1043D00001020304060708090000000000000000B5
:1043E00000000000000000000000000000000000CD
:1043F000000000000000CDAB000000000000000045
:1044000000000000000000000000000000000000AC
:10441000000000000000000000000000000000009C
:10442000000000000000000000000000000000008C
:1044300000A24A0400000000000000000102030482
:04444000060708095A
:04000005080001519D
:00000001FF
